:020000040000FA
:02000000002BD3
:100010004934433453343134303430344C3469341B
:100020003E343E34563431342E3431343C343C3456
:10003000A0148519A30A1C28A40A0319A40385196E
:10004000A30A0000C9208519A30A260885002208F2
:10005000A10000008519A30AA10085191828A0187D
:100060003628A3018519A30A35281F282308A800CC
:1000700003302402031CA017031CA81BA013C920D3
:100080004128260885002208A1000000A1000830B0
:1000900024020318A017A4018030A802BA30280255
:1000A0000318A017A01B88282908A807A80CC92096
:1000B0005928260885002208A1002808C720A50085
:1000C0003F39A20003192611251B7228A6106828A3
:1000D000C9201930AB00260885002208A100031DA5
:1000E00026157B28261126088500AB0B7B28AB0A3A
:1000F000A614260885002808A900AA08031DAA033B
:100100008128822883286400A010A301C920252803
:100110008928C9200000A013260885002208A10014
:100120009128A100AA0A32302A02031C8028261135
:10013000A6102612A616260885002F2B2611261299
:1001400026088500A614260885002F2BA101051579
:10015000A928AA28AB28AC28AD28AE280000051194
:100160003C30A2006400A20BB2283C30A200640024
:10017000A20BB728A10BA72800348030A100F930CA
:10018000A4006400A40BC128A10BBF2800348A146A
:1001900082002608FB39191F9E288519A30AA1038E
:1001A00003198500191F9E288519A30AA1030319A5
:1001B0008500191F9E288519A30AA103031985002C
:1001C000191F9E288519A30AA10303198500191F69
:1001D0009E288519A30AA10303198500191F9E28CB
:1001E0008519A30AA10303198500191F9E288519E3
:1001F000A30AA10303198500191F9E288519A30AC4
:10020000A10303198500191F9E288519A30AA103BC
:1002100003198500191F9E288519A30AA103031934
:100220008500191F9E288519A30AA10303198500BB
:10023000191F9E288519A30AA10303198500191FF8
:100240009E288519A30AA10303198500191F9E285A
:100250008519A30AA10303198500191F9E28851972
:10026000A30AA10303198500191F9E288519A30A53
:10027000A10303198500191F9E288519A30AA1034C
:1002800003198500191F9E288519A30AA1030319C4
:100290008500191F9E288519A30AA103031985004B
:1002A000191F9E288519A30AA10303198500191F88
:1002B0009E288519A30AA10303198500191F9E28EA
:1002C0008519A30AA10303198500191F9E28851902
:1002D000A30AA10303198500191F9E288519A30AE3
:1002E000A10303198500191F9E288519A30AA103DC
:1002F00003198500191F9E288519A30AA103031954
:100300008500191F9E288519A30AA10303198500DA
:10031000191F9E288519A30AA10303198500191F17
:100320009E288519A30AA10303198500191F9E2879
:100330008519A30AA10303198500191F9E28851991
:10034000A30AA10303198500191F9E288519A30A72
:10035000A10303198500191F9E288519A30AA1036B
:1003600003198500191F9E288519A30AA1030319E3
:100370008500191F9E288519A30AA103031985006A
:10038000191F9E288519A30AA10303198500191FA7
:100390009E288519A30AA10303198500191F9E2809
:1003A0008519A30AA10303198500191F9E28851921
:1003B000A30AA10303198500191F9E288519A30A02
:1003C000A10303198500191F9E288519A30AA103FB
:1003D00003198500191F9E288519A30AA103031973
:1003E0008500191F9E288519A30AA10303198500FA
:0203F0000034D7
:10040000403440344034403440344034403440344C
:10041000403440344034403440344034403440343C
:10042000403440344034403440344034403440342C
:10043000403440344034403440344034403440341C
:10044000403440344034403440344034403440340C
:100450004034403440340034003400340334053434
:100460000634073409340A340A340B340C340D349E
:100470000E340E340F34103410341134123412345C
:100480001334133414341534153416341634173425
:100490001734183418341934193419341A341A34F6
:1004A0001B341B341C341C341C341D341D341E34CA
:1004B0001E341E341F341F342034203420342134A1
:1004C000213421342234223422342334233423347B
:1004D0002434243424342534253425342634263455
:1004E0002634273427342734283428342834283431
:1004F0002934293429342A342A342A342B342B340D
:100500002B343F343F343F343F343F343F343F3467
:100510003F343F343F343F343F343F343F343F3443
:100520003F343F343F343F343F343F343F343F3433
:100530003F343F343F343F343F343F343F343F3423
:100540003F343F343F343F343F343F343F343F3413
:100550003F343F343F343F343F343F343F343F3403
:100560003F343F343F343F343F343F343F343F34F3
:100570003F343F343F343F343F343F343F343F34E3
:100580003F343F343F343F343F343F343F343F34D3
:100590003F343F343F343F343F343F343F343F34C3
:1005A0003F343F343F343F343F343F343F343F34B3
:1005B0003F343F343F343F343F343F343F343F34A3
:1005C0003F343F343F343F343F343F343F343F3493
:1005D0003F343F343F343F343F343F343F343F3483
:1005E0003F343F343F343F343F343F343F343F3473
:1005F0003F343F343F343F343F343F343F343F3463
:10060000850183160930850001309F00FF2390008B
:100610008230990083121E30990064008101DF301E
:100620008316810083126400DC30831681008312FC
:100630006400A101A40164001D2B1E2B1F2B202B85
:10064000212B222B232BA40B1B2BA10B1A2B2015A8
:10065000191B2F2B20118316A530990083126400DB
:10066000191F2F2B6400191F2F2B851D322B191FCB
:100670002F2B8519372B1930A700A3016400191FF0
:100680002F2B851D3F2BA30A03192F2B0000851943
:10069000432B64008030A3022B3023020318322B3B
:1006A000A70B3D2B201D562BA620BD20A620BD202C
:1006B000A620851D592B85195B2BA201A301A4013E
:1006C000A901AA01A013A0102010A60126161F2818
:0207FE0048347D
:02400E00DC3F95
:00000001FF
